:020000020000FC
:02000000ACC092
:02000C0004C02E
:1000140021C00FB61F9381FF03C07A9509F4B39AE8
:1000240080FF05C0459B03C055D08260772710B37D
:1000340015FF82FF0AC081FF02C04CD006C080FFBA
:1000440002C048D002C041D000C015FB82F91F9104
:100054000FBE1895189510E012B911E019B98599D9
:1000640008C010E012B91BE019B9C09A859BFECFF5
:10007400C09810E01BB918E11AB916E013B9089535
:100084005D9BFECF4CB908955F9BFECF4CB10895A4
:100094002FEF2A95F1F71A95D9F70895332718E029
:1000A400F0E0331F10F4C69A01C0C698FF0FB5994B
:1000B400F160C79A26E02A95F1F7C79823E02A95BC
:1000C400F1F71A9571F73F2F08958D7F9698C39A8B
:1000D400816008958D7F8E7F969AC39808951DED53
:1000E40017BBC798C49A1FEFD3DFC4981FEFD0DFA4
:1000F4003CEAD5DF33E5D3DF0032B8F00023AAF0C1
:10010400A0E2CCDF333599F030E0C9DFC79A26E0AE
:100114002A95F1F7C79823E02A95F1F73CEABFDF67
:1001240033E5BDDFAA9569F702C030E0B8DF30E0FF
:10013400B6DF10E1ADDF089541E4A2DF46E5A0DFBC
:1001440042E59EDF40E29CDF49E49ADF43E598DF25
:1001540040E596DF08951FED1DBF8827469A0000ED
:1001640010E011BB8E9A959A969A11271BBFC49AD8
:100174001DE017BB10E018BB6EDF439A13E013BFFA
:1001840012E019BF789480DF4B31E9F3443519F458
:100194007BDF042F57C1433511F4CEDFF4CF46354E
:1001A40029F442E36DDF43E36BDFEDCF463729F4F7
:1001B40041E666DF40E664DFE6CF443749F545E5CE
:1001C4005FDF46E55DDF43E15BDF40E259DF48E2A4
:1001D40057DF48E355DF48E453DF4CE451DF44E3A1
:1001E4004FDF40E34DDF4CE64BDF48E649DF45E6B1
:1001F40047DF40E645DF44E643DF42E741DF41E4D1
:100204003FDF42E43DDF43E23BDF40E039DFBBCF89
:10021400403719F443E534DFB6CF413619F449E5E4
:100224002FDFB1CF483711F4C09A0CC1493711F40C
:10023400C09808C1053529F1063519F1033109F1D2
:100244000032F9F00832E9F00833D9F00834C9F083
:100254000C34B9F00433A9F0003399F00C3689F06A
:10026400083679F0053669F0003659F0043649F05D
:10027400023739F0023429F0013419F0033209F05D
:10028400DEC0403541F4C29A8860459B02C0877F36
:100294001CDF25DFD7C0433471F4F6DE38E4FFDE1B
:1002A400362FFDDE352FFBDE342FF9DE11E0222759
:1002B400510F621F0BC04336B9F4E6DE30E4EFDEC3
:1002C400362FEDDE352FEBDE342FE9DE013459F025
:1002D400053649F0023439F0003629F0043619F0B5
:1002E400023710E2D5DEAEC0423599F438E2D7DEEB
:1002F400362FD5DE352FD3DED1DE432FC1DE30E2FB
:10030400CEDE362FCCDE352FCADEC8DE432FB8DE74
:1003140024C0413429F4B8DE642FB6DE542F92C0D1
:10032400443481F4B1DE30ECBADE362FB8DE352F3A
:10033400B6DE342FB4DE10E2ABDE11E02227510F1B
:10034400621F80C0443671F430EAA9DE362FA7DE7E
:10035400352FA5DEA3DE432F93DE11E02227510FB4
:10036400621F11CF4C3449F41DE017BBC49AC298E4
:1003740083FD02C081FFAEDE65C0453659F43CEA18
:100384008EDE30E88CDE34E08ADE30E088DE10E396
:100394007FDE58C04C3671F477DE3CEA80DE342FC1
:1003A4003670306E7CDE30E07ADE30E078DE10E3EA
:1003B4006FDE48C0433789F4B2E005D0B1E003D022
:1003C400B0E001D0E0CE30E36ADE30E068DE3B2FFF
:1003D40066DE64DE432F54DE08954D3659F43CE462
:1003E4005EDE362F5CDE352F5ADE30E058DE1FEF3E
:1003F4004FDE28C04A3359F447DEC42F45DED42FDC
:1004040043DEE42F442710D01FEF42DE1BC04E32E0
:10041400B1F43ADEC42F38DED42F36DEE42F34DED6
:1004240003D01FEF35DE0EC03C2F39DE3D2F37DE03
:100434003E2F35DE342F33DE4F2F22DE08954FE377
:100444001FDEA1CE4DE01CDE9ECE0000133029F04D
:0C045400000000001A951330E9F708952D
:00000001FF
